:0A00000075817F7401F58F02000E78
:10000B0002023FC229C2287400900010F090001128
:10001B00F0900012F0900013F0900014F074009028
:10002B000016F07401900017F07402900018F07431
:10003B0003900019F0740490001AF0740590001BE3
:10004B00F0740690001CF0740790001DF07408907B
:10005B00001EF0740990001FF0740A900020F074D9
:10006B000B900021F07400900031F0900032F09072
:10007B000033F0900034F0900035F0740290002FB4
:10008B00F07402900030F090003779FF7400F0A309
:10009B00D9FA90013679FF7400F0A3D9FA900237A0
:1000AB0079FF7400F0A3D9FA90033679CD7400F080
:1000BB00A3D9FA120EBF7564FF7565FF7566FF75E0
:1000CB00460075470075710075680075720075699B
:1000DB0000C208C2097540007541007542007543A6
:1000EB0000754C00754D007570027548FF75490A17
:1000FB0085483C85493D754A7F754B01854A44854A
:10010B004B45755500D226C2C175A012C2B1C2B300
:10011B00C2B4C2B5C2B6C281C2B2C28412069712B1
:10012B0006B61206D51206F412081A75597F755ABF
:10013B007F755B7F755D00755E00755F001201EF6B
:10014B001205921205ED12219C75730075740175E1
:10015B0072001216EA121F3A121F45D20FD22CC28E
:10016B002E12239B12081A12242D122559121F3AF4
:10017B00121F451208BD120B0E120EDC12155D126A
:10018B001575121CF5121CDA1223D002016C856056
:10019B0090C2A7C2C0D2C022856290D2A7C2C0D2E1
:1001AB00C022C285C281C2B2C284E56479081392AF
:1001BB0083C285D285D9F7D2810000C281E56579EA
:1001CB0008139283C285D285D9F7D2B20000C2B28E
:1001DB00E5667908139283C285D285D9F7D284005C
:1001EB0000C28422758790758922758DFC758BFCF6
:1001FB00759850C299C298758C38758A38753906BE
:10020B00753A04753B0590FF9C8582CA8583CB8527
:10021B0082CC8583CDC200C201D28CD2A9D2AF22AF
:10022B00783279320000D9FCD8F822780A790FD9C4
:10023B00FED8FA22C2AFC0E0C0D0E5F0C0E0E58244
:10024B00C0E0E583C0E0E575C0E043D0081206D5F9
:10025B001225051225191211B9D544107544FFD575
:10026B00450A854A44854B45D223D227122447128F
:10027B00247E121B0A12245D1203E012043E122587
:10028B002D12249DD5392A753906B20330030F126E
:10029B00071312067F1201991201A30202AC12017D
:1002AB00ADD53A0D753A04303307D53B04D2A0C215
:1002BB0033D0E0F575D0E0F583D0E0F582D0E0F5F2
:1002CB00F0D0D0D0E0D2AF32E54FB4021130240ED3
:1002DB00D287C282054DD2A2121F7702205C22E583
:1002EB005575F001241084E5F0B40014E54FB4000B
:1002FB0006755680020370B40206755680020370B1
:10030B0022E55575F001241084E5F0B4000BE54FA0
:10031B00B4000675565002037022E55575F00224A1
:10032B001084E5F0B4000BE54FB4000675562202BD
:10033B00037022E55575F004241084E5F0B4000B2E
:10034B00E54FB4000675561002037022E55575F0A3
:10035B0008241084E5F0B4000BE54FB40006755685
:10036B000702037022200C0C302409D2B6C280D2B3
:0E037B00041211DBD21B85525022E55A75F098
:100389001E84B40403020357B4050302033EB406F2
:1003990003020325B4070302030CB4080302030C88
:1003A90022E559B40F030203B4500574010203C2D4
:1003B900C3940F8556F0842401F55222E559B40FF0
:1003C900030203CF500574010203DDC3940F855660
:1003D900F0842401F55322D53C0302040DD53C03D6
:1003E90002040DD53C0302040DD53C0302040DD5CE
:1003F9003C0302040DD53C0302040DD53C03020461
:100409000DD53C0DD53D0A85483C85493D054FD262
:10041900013001201202D3301B0FD5500CC21B2012
:100429002007302404C2B6D280121D7E1203851221
:1004390003AAC20122D53E0302045FD53E0302048A
:100449005FD53E0302045FD53E0302045FD53E0338
:1004590002045FD53E0DD53F0A85483E85493F05D3
:100469004ED20030000B12047B1205731203C5C271
:100479000022201A0122D5500CC21A20200730244C
:1004890004C2B6D28022E55575F002241084E5F045
:10049900B40014E54EB4000675568002055EB40238
:1004A9001475568002055EB4010BE54EB40106755C
:1004B900568002055E22E55575F004241084E5F0A6
:1004C900B4010BE54EB4002275567802055EB402FC
:1004D9000BE54EB4011475567802055EB4030BE5BD
:1004E9004EB4020675567802055E22E55575F00888
:1004F900241084E5F0B4010BE54EB40022755630A2
:1005090002055EB4030BE54EB402147556300205BC
:100519005EB4060BE54EB4010675563002055E223F
:10052900E55575F010241084E5F0B4010BE54EB4DF
:10053900002275561502055EB4060BE54EB401148A
:1005490075561502055EB40B0BE54EB402067556D9
:100559001502055E22200C0C302409D2B6C280D2C5
:10056900041211DBD21A85535022E55A75F01E8404
:10057900B400030204BFB401030204BFB4020302BE
:1005890004F4B40303020529227564F712023675CF
:1005990064DF1202367564FF7565F71202367565F8
:1005A900FD1202367565FF7566DF1202367566FD46
:1005B90012023675667F1202367566FF75647F1200
:1005C90002367564FD1202367564FF7565DF120225
:1005D9003675657F1202367565FF7566F712023644
:1005E9007566FF227564F31202367564CF120236FE
:1005F9007564FF7565F31202367565FC120236756E
:1006090065FF7566CF1202367566FC12023675668D
:100619003F1202367566FF75643F1202367564FC37
:100629001202367564FF7565CF12023675653F1281
:1006390002367565FF7566F31202367566FF227517
:1006490064001201AD7564001201AD7564001201F8
:10065900AD7564551201AD7564001201AD75640084
:100669001201AD7564001201AD7566551201AD75C3
:0D06790065001201AD22E546B400050546FE
:10068600020697B4010505460206B675460002063F
:10069600F474FE7908339283D285C285D9F7C2B73E
:1006A600D2B77908A2A133D2A6C2A6D9F7F56A2293
:1006B60074FD7908339283D285C285D9F7C2B7D241
:1006C600B77908A2A133D2A6C2A6D9F7F56B2274D0
:1006D600FB7908339283D285C285D9F7C2B7D2B7E0
:1006E6007908A2A133D2A6C2A6D9F7F56C2274F76F
:1006F6007908339283D285C285D9F7C2B7D2B77942
:1007060008A2A133D2A6C2A6D9F7F56D22E547B451
:1007160000050547020743B40105054702076AB409
:100726000205054702078CB4030505470207AEB468
:10073600040505470207D87547000207FCC2A3C295
:1007460086C2B0D2A57914D9FEC2A57908C2A6D2AE
:10075600A6A2A433D9F7C2A6F55D20340122C2347D
:100766001214DE22D2A3C286C2B0D2A57914D9FE53
:10077600C2A57908C2A6D2A6A2A433D9F7C2A630CA
:10078600280122F55922C2A3D286C2B0D2A5791475
:10079600D9FEC2A57908C2A6D2A6A2A433D9F7C2A9
:1007A600A630280122F55A22D2A3C286D2B0D2A5FB
:1007B6007914D9FEC2A57908C2A6D2A6A2A433D9B5
:1007C600F7C2A63028030207D1F55B30290122F5CE
:1007D6005C22D2A3D286C2B0D2A57914D9FEC2A514
:1007E6007908C2A6D2A6A2A433D9F7C2A630350389
:1007F600C23522F55E22C2A3C286D2B0D2A5791432
:10080600D9FEC2A57908C2A6D2A6A2A433D9F7C238
:10081600A6F55F2212084412085212083612086022
:1008260012086E12087C12088A12089B1208AC2263
:10083600E56C30E4012220E60122756E0022E56CAB
:1008460020E4012220E60122756E0122E56C20E4F7
:10085600012230E60122756E0222E56B30E30122A9
:1008660020E50122756F0022E56B20E3012220E5D9
:100876000122756F0122E56B20E3012230E501229A
:10088600756F0222E56D30E6012220E50122740132
:1008960090002FF022E56D20E6012220E50122746A
:1008A6000290002FF022E56D20E6012230E50122BC
:1008B600740490002FF022E56F7017C22EC22DD25D
:1008C6000F1208D9120A1212093E120B081209E574
:1008D600D22C22302907900031E00208E5E55CB40D
:1008E60078030208F050030208F2747975F0178451
:1008F600B4000C756700C2B1C2B3C2B5C2B422B4AB
:10090600010C756701D2B1C2B3C2B5C2B422B4023A
:100916000C756702C2B1D2B3C2B5C2B422B4030C1D
:10092600756703C2B1C2B3D2B5C2B422756704C239
:10093600B1C2B3C2B5D2B422E56775F030A425685A
:10094600F56022E56BF430E009757101D22A1209CF
:10095600EE2230E109757100D22A1209EE2230E248
:1009660009757102D22A1209EE2230E60975710361
:10097600D22A1209EE22E56AF430E009757106D230
:100986002A1209EE2230E109757109D22A1209EEFE
:100996002230E20975710AD22A1209EE2230E309E1
:1009A600757107D22A1209EE2230E40975710BD24D
:1009B6002A1209EE2230E509757108D22A1209EECB
:1009C6002230E609757105D22A1209EE2230E709AE
:1009D600757104D22A1209EE22C22A1209EE2220C9
:1009E6002A03D2A022C2A022E571202A05C2E7F579
:0E09F6006922D2E7F56922900032E020E7077F
:100A0400C22AC2E7F57122D22AC2E7F5712230293F
:100A1400061209FD020A21120949020A21E571B4EC
:100A2400011075680412093E75647F7565FF75666B
:100A3400FF22B4001075680012093E7564F77565ED
:100A4400FF7566FF22B4021075680812093E7564CA
:100A5400DF7565FF7566FF22B4031075680C120913
:100A64003E7564FD7565FF7566FF22B406107568F2
:100A74001812093E7564FF7565DF7566FF22B409B7
:100A84001075682412093E7564FF7565FF7566FD6F
:100A940022B40A1075682812093E7564FF7565FF53
:100AA4007566F722B4071075681C12093E7564FF59
:100AB4007565FF7566DF22B40B1075682C12093E4C
:100AC4007564FF7565FF75667F22B408107568202C
:100AD40012093E7564FF75657F7566FF22B40510C3
:100AE40075681412093E7564FF7565FD7566FF220D
:100AF400B4041075681012093E7564FF7565F775C6
:100B040066FF2222E571120CE822E56F7003D20F12
:100B140022E56EB40212D22CC22EC22D300F051261
:100B24000EB3C20F120CCB22D20F22E55EB43803EF
:100B3400020B395003790022B43C03020B445003E6
:100B4400790122B44103020B4F5003790222B445C8
:100B540003020B5A5003790322B44A03020B655073
:100B640003790422B44E03020B705003790522B4B6
:100B74005303020B7B5003790622B45703020B86FE
:100B84005003790722B45C03020B915003790822C5
:100B9400B46003020B9C5003790922B46503020B71
:100BA400A75003790A22B46A03020BB25003790BEB
:100BB40022790B22120B2FE9900033F0120CC6128B
:100BC4000EB322900033E0F575120B2FE9B57503CF
:100BD400020BF1E55EB43404120BB8225003020B8D
:100BE400F1B46B03020BF15004120BB822E56BF461
:100BF40030E00E200E51D20E7901120CC6120EB343
:100C04002230E10E200E40D20E7900120CC6120ED4
:100C1400B32230E20E200E2FD20E7902120CC6122D
:100C24000EB32230E60E200E1ED20E7903120CC62D
:100C3400120EB322E56AF430E00E200E0AD20E79C9
:100C440006120CC6120EB32230E10E200E70D20E24
:100C54007909120CC6120EB32230E20E200E5FD2B6
:100C64000E790A120CC6120EB32230E30E200E4E79
:100C7400D20E7907120CC6120EB32230E40E200EE7
:100C84003DD20E790B120CC6120EB32230E50E20A3
:100C94000E2CD20E7908120CC6120EB32230E60EB8
:100CA400200E1BD20E7905120CC6120EB32230E7A9
:100CB4000E200E0AD20E7904120CC6120EB322C2F2
:100CC4000E228969897122302911900032E0C2E72D
:100CD400B5710122D20FF571020EB3020BC7E57193
:100CE400120CE822B4010A75647F7565FF7566FF0E
:100CF40022B4000A7564F77565FF7566FF22B402B5
:100D04000A7564DF7565FF7566FF22B4030A7564AE
:100D1400FD7565FF7566FF22B4060A7564FF756587
:100D2400DF7566FF22B4090A7564FF7565FF756691
:100D3400FD22B40A0A7564FF7565FF7566F722B46F
:100D4400070A7564FF7565FF7566DF22B40B0A75C3
:070D540064FF7565FF756681
:100D5B007F22B4080A7564FF75657F7566FF22B440
:100D6B00050A7564FF7565FD7566FF22B4040A7587
:100D7B0064FF7565F77566FF2222B4010A75643F3F
:100D8B007565FF7566FF22B4000A7564F37565FF20
:100D9B007566FF22B4020A7564CF7565FF7566FF31
:100DAB0022B4030A7564FC7565FF7566FF22B406F1
:100DBB000A7564FF7565CF7566FF22B4090A756401
:100DCB00FF7565FF7566FC22B40A0A7564FF7565CD
:100DDB00FF7566F322B4070A7564FF7565FF7566C8
:100DEB00CF22B40B0A7564FF7565FF75663F22B49D
:100DFB00080A7564FF75653F7566FF22B4050A75B1
:100E0B0064FF7565FC7566FF22B4040A7564FF7593
:100E1B0065F37566FF2222B40109E564C2E7D2E6E9
:100E2B00F56422B40009E564C2E3D2E2F56422B4AE
:100E3B000209E564C2E5D2E4F56422B40309E56472
:100E4B00C2E1D2E0F56422B40609E565C2E5D2E45D
:100E5B00F56522B40909E566C2E1D2E0F56622B474
:100E6B000A09E566C2E3D2E2F56622B40709E56634
:100E7B00C2E5D2E4F56622B40B09E566C2E7D2E619
:100E8B00F56622B40809E565C2E7D2E6F56522B43A
:100E9B000509E565C2E1D2E0F56522B40409E56513
:100EAB00C2E3D2E2F5652222120EBF1210FEE571EB
:100EBB00120E2222790C90002205A2900016E0A3BC
:100ECB0020E70605A2F0A305A2D9F305A27480F0D2
:100EDB0022E56F700122E56EB40116D22CC22F12DF
:100EEB001723121706202E09120EFD120FC7120E12
:100EFB00BF22E56BF430E00D200D4CD20D900017A6
:100F0B00E0B2E7F02230E10D200D3CD20D9000163F
:100F1B00E0B2E7F02230E20D200D2CD20D9000183C
:100F2B00E0B2E7F02230E60D200D1CD20D90001937
:100F3B00E0B2E7F022E56AF430E00D200D09D20DA6
:100F4B0090001CE0B2E7F02230E10D200D6DD20DC8
:100F5B0090001FE0B2E7F02230E20D200D5DD20DC4
:100F6B00900020E0B2E7F02230E30D200D4DD20DC2
:100F7B0090001DE0B2E7F02230E40D200D3DD20DC4
:100F8B00900021E0B2E7F02230E50D200D2DD20DBF
:100F9B0090001EE0B2E7F02230E60D200D1DD20DC1
:100FAB0090001BE0B2E7F02230E70D200D0DD20DC3
:100FBB0090001AE0B2E7F022C20D2222900017E057
:100FCB0020E70BE564C2E7C2E6F564020FE1E564D6
:100FDB00D2E7D2E6F564900016E020E70BE564C299
:100FEB00E3C2E2F564020FFBE564D2E3D2E2F564FF
:100FFB00900018E020E70BE564C2E5C2E4F564025B
:10100B001015E564D2E5D2E4F564900019E020E711
:10101B000BE564C2E1C2E0F56402102FE564D2E196
:10102B00D2E0F56490001CE020E70BE565C2E5C259
:10103B00E4F565021049E565D2E5D2E4F56590006B
:10104B001FE020E70BE566C2E1C2E0F56602106324
:10105B00E566D2E1D2E0F566900020E020E70BE5F3
:0C106B0066C2E3C2E2F56602107DE56695
:10107700D2E3D2E2F56690001DE020E70BE566C2F9
:10108700E5C2E4F566021097E566D2E5D2E4F566B7
:10109700900021E020E70BE566C2E7C2E6F56602AD
:1010A70010B1E566D2E7D2E6F56690001EE020E7CC
:1010B7000BE565C2E7C2E6F5650210CBE565D2E749
:1010C700D2E6F56590001BE020E70BE565C2E1C2BB
:1010D700E0F5650210E5E565D2E1D2E0F56590003F
:1010E7001AE020E709E565C2E3C2E2F56522E56596
:1010F700D2E3D2E2F565227564FF7565FF7566FF79
:10110700900022E0FAE0F92571C39AB40C030211AA
:101117001D5003021120C3940C121129A3E930E7D3
:10112700E422B40109E564C2E7C2E6F56422B4002B
:1011370009E564C2E3C2E2F56422B40209E564C2C8
:10114700E5C2E4F56422B40309E564C2E1C2E0F54F
:101157006422B40609E565C2E5C2E4F56522B4096F
:1011670009E566C2E1C2E0F56622B40A09E566C28E
:10117700E3C2E2F56622B40709E566C2E5C2E4F513
:101187006622B40B09E566C2E7C2E6F56622B40833
:1011970009E565C2E7C2E6F56522B40509E565C25A
:1011A700E1C2E0F56522B40408E565C2E3C2E2F5F1
:1011B7006522E56FB4011CE56C30E503C2252220EA
:1011C7002511D225D234D235753A03754704C203A7
:1011D70075390622300419C204202014E56FB402C1
:1011E7000FD234D235753A03754704C203753906F1
:1011F70022E55DB402030212025003790022B4060D
:101207000302120D5003790122B40A030212185087
:1012170003790222B40F030212235003790322B485
:10122700130302122E5003790422B4180302123951
:101237005003790522B41D03021244500379062294
:10124700B4210302124F5003790722B42503021277
:101257005A5003790822B42A030212655003790908
:1012670022B42E030212705003790A22B433030208
:10127700127B5003790B22790B22E55DB437030209
:10128700128B5003790022B43C0302129650037963
:101297000122B440030212A15003790222B445038C
:1012A7000212AC5003790322B449030212B7500368
:1012B700790422B44E030212C25003790522B452B4
:1012C700030212CD5003790622B457030212D850F5
:1012D70003790722B45B030212E35003790822B4AF
:1012E70060030212EE5003790922B464030212F973
:1012F7005003790A22B468030213045003790B22BE
:10130700790B22E55DB46D030213145003790022B3
:10131700B4710302131F5003790122B47603021339
:101327002A5003790222B47A030213355003790352
:1013370022B47E030213405003790422B4830302CC
:10134700134B5003790522B48703021356500379D0
:101357000622B48C030213615003790722B4900369
:1013670002136C5003790822B495030213775003D4
:10137700790922B499030213825003790A22B49E91
:101387000302138D5003790B22790B22E55DB4A27A
:101397000302139D5003790022B4A7030213A85038
:1013A70003790122B4AB030213B35003790222B4C9
:1013B700B0030213BE5003790322B4B4030213C966
:1013C7005003790422B4B9030213D45003790522D8
:1013D700B4BD030213DF5003790622B4C10302131D
:0E13E700EA5003790722B4C6030213F550033F
:1013F500790822B4CA030214005003790922B4CF34
:101405000302140B5003790A22B4D40302141650B4
:1014150003790B22790B22E55DB4D803021426501B
:1014250003790022B4DC030214315003790122B49C
:10143500E10302143C5003790222B4E50302144788
:101445005003790322B4EA030214525003790422AB
:10145500B4EE0302145D5003790522B4F3030214BC
:10146500685003790622B4F7030214735003790711
:1014750022B4FC0302147E5003790822B4FE030251
:1014850014895003790922790A22E55DB4330302F0
:10149500149950091211F889757400FB22B4680378
:1014A5000214AA500912128189757401FB22B49E97
:1014B500030214BB500912130A89757402FB22B486
:1014C500D4030214CC500912139389757403FB22BB
:1014D50012141C89757404FB2212148F7A00900073
:1014E50022E020E70DB575030214F85006A3FA02B1
:1014F50014E6EA2571F9BB0424B40A030215224057
:101505001C7A00900022E020E70D2571B40A06E060
:10151500FAA302150B40F8EA2571021523E975F0C7
:1015250004A4F9EB75F030A4FAE92AF560EB12088A
:10153500F612154822900036E0F560EB1208F61217
:10154500154822E56F6010E560B56101228560618F
:10155500C2A0D233753B0222E56F700122E56EB45D
:10156500000DC22EC22D121A0F1216701215A722C7
:10157500E56F700122E56EB40115121A0F30300FB8
:101585001216EA120EFD120FC7120EBFC23022B498
:10159500020F121A0F3031091216EA120EB3C231B8
:1015A5002222202C0122E573120D85E574120E22EC
:1015B500C22CE56F700122E56EB40006302F0312D0
:1015C50016EA22E56BF430E114E572C2E0C2E1C22D
:1015D500E2C2E3F572757300D22CD22F2230E214E9
:1015E500E572D2E0C2E1C2E2C2E3F572757302D2DE
:1015F5002CD22F22E56AF430E114E572D2E0C2E183
:10160500D2E2C2E3F572757309D22CD22F2230E3F0
:1016150014E572C2E0C2E1D2E2C2E3F57275730766
:10162500D22CD22F2230E414E572C2E0D2E1D2E20C
:10163500C2E3F57275730BD22CD22F2230E614E576
:1016450072D2E0D2E1C2E2C2E3F572757305D22C23
:10165500D22F2230E714E572C2E0D2E1C2E2C2E342
:10166500F572757304D22CD22F2222E56BF430E08B
:1016750014E572C2E4C2E5C2E6C2E7F5727574010B
:10168500D22CD22F2230E614E572D2E4C2E5C2E6AE
:10169500C2E7F572757403D22CD22F22E56AF430B5
:1016A500E014E572C2E4D2E5C2E6C2E7F5727574EC
:1016B50006D22CD22F2230E514E572D2E4D2E5C24F
:1016C500E6C2E7F572757408D22CD22F2230E214E7
:1016D500E572C2E4C2E5D2E6C2E7F57275740AD2D4
:1016E5002CD22F2222E572C2E0C2E1C2E2C2E3C4DB
:1016F500B4040712214F120EBF2212217A120EBF17
:1017050022E56C30E303C22B22202B11D22B202D96
:1017150005D22ED22D22C22E12211FC22D22202EFD
:101725000122E572C2E4C2E5D2E6C2E7F57275743C
:101735000A1215C81215A722900034E0F575121A81
:101745000FE9B57503021767E55FB43404121A0F84
:10175500225003021767B454030217675004121A84
:0E1765000F221215C822E55FB4370302177574
:1017730050077401900035F022B43C0302178450E3
:10178300077402900035F022B44003021793500708
:101793007403900035F022B445030217A250077476
:1017A30004900035F022B449030217B150077405C1
:1017B300900035F022B44E030217C0500774069010
:1017C3000035F022B452030217CF5007740790007C
:1017D30035F02222E55FB457030217E15007740185
:1017E300900035F022B45B030217F05007740290A7
:1017F3000035F022B460030217FF50077403900012
:1018030035F022B4640302180E50077404900035B7
:10181300F022B4680302181D50077405900035F0D8
:1018230022B46D0302182C50077406900035F02281
:10183300B4710302183B50077407900035F022225D
:10184300E55FB4760302184D50077401900035F03C
:1018530022B47A0302185C50077402900035F02218
:10186300B47E0302186B50077403900035F022B462
:10187300830302187A50077404900035F022B4876A
:101883000302188950077405900035F022B48C03C5
:1018930002189850077406900035F022B4900302A2
:1018A30018A750077407900035F02222E55FB4951E
:1018B300030218B950077401900035F022B499035C
:1018C3000218C850077402900035F022B49E030238
:1018D30018D750077403900035F022B4A2030218FE
:1018E300E650077404900035F022B4A7030218F5FC
:1018F30050077405900035F022B4AB03021904506D
:10190300077406900035F022B4B003021913500790
:101913007407900035F02222E55FB4B40302192561
:1019230050077401900035F022B4B9030219345002
:10193300077402900035F022B4BD03021943500727
:101943007403900035F022B4C10302195250077496
:1019530004900035F022B4C60302196150077405E0
:10196300900035F022B4CA03021970500774069030
:101973000035F022B4CF0302197F5007740790009B
:1019830035F02222E55FB4330122500122B4520321
:10199300021998501312176BE572C2E4C2E5C2E64E
:1019A300C2E7F57275740122B471030219B35013BF
:1019B3001217D7E572D2E4C2E5C2E6C2E7F5727543
:1019C300740322B490030219CE5013121843E57224
:1019D300C2E4D2E5C2E6C2E7F57275740622B4B07A
:1019E300030219E950131218AFE572D2E4D2E5C22B
:1019F300E6C2E7F5727574082212191BE572C2E498
:101A0300C2E5D2E6C2E7F57275740A22121987900D
:101A13000034E0F576900035E0B5760EE56F7001A1
:101A230022E56EB400031215C822D22F900035E0D0
:101A3300900034F0B40103021A3F5016E572C2E07D
:101A4300C2E1C2E2C2E3F572757300D22CD231D285
:101A53003022B40203021A5D5016E572D2E0C2E1ED
:101A6300C2E2C2E3F572757302D22CD231D23022B4
:101A7300B40303021A7B5016E572C2E0D2E1C2E25C
:101A8300C2E3F572757304D22CD231D23022B4047E
:101A930003021A995016E572D2E0D2E1C2E2C2E320
:101AA300F572757305D22CD231D23022B4050302FC
:101AB3001AB75016E572C2E0C2E1D2E2C2E3F57290
:101AC300757307D22CD231D23022B40603021AD551
:101AD3005016E572D2E0C2E1D2E2C2E3F572757349
:0E1AE30009D22CD231D23022B40703021AF3FA
:101AF1005016E572C2E0D2E1D2E2C2E3F57275732B
:101B01000BD22CD231D230222230231A054C121C96
:101B1100A3121B46121B7F121B2A121B6E121C5191
:101B2100121CB7121D1BC22322E54C75F01824604C
:101B310084E5F0B40C06202402C28222B400052000
:101B41002402D28222E54C75F006246084E5F0B4CB
:101B5100030C202408D287121F7702205C22B400D4
:101B61000B202408C287121F7702205C22E54CB4A7
:101B7100600B754C00202405C2A2121F50222024A4
:101B81000BE54CB4000122B40302D2A222E54C754C
:101B9100F030246084E5F0B400097557087563607E
:101BA100021C8E22E54C75F018246084E5F0B40027
:101BB1000975570F756360021C8E22E54C75F00C98
:101BC100246084E5F0B4000975571E756360021C3A
:101BD1008E22E54C75F006246084E5F0B4000975A9
:101BE100573C756360021C8E22E54C75F00324603E
:101BF10084E5F0B40009755778756360021C8E2284
:101C0100E54C75F020246084E5F0B4000675570AB0
:101C1100021C8E22E54C75F010246084E5F0B400BE
:101C210006755714021C8E22E54C75F00824608459
:101C3100E5F0B40006755728021C8E22E54C75F0BC
:101C410004246084E5F0B40006755750021C8E220E
:101C5100E55A75F01E84B40003021C3DB401030271
:101C61001C29B40203021C15B40303021C01B404B1
:101C710003021B8EB40503021BA5B40603021BBCA1
:101C8100B40703021BD3B40803021BEA22200C0C85
:101C9100202409D2B6C280D2041211DBD21C855491
:101CA1005122201C0122D5510CC21C2020072024C6
:101CB10004C2B6D28022E559B40F03021CC15005FB
:101CC1007401021CCFC3940F8557F0842401F5548D
:101CD100E557B4800375540122E55975F00484B4C5
:101CE1000005D20CC22022B43F05C20CD22022C270
:101CF1000CC22022E55BB4A003021D09500A122385
:101D01007475F002A4021D18B4C803021D17500611
:101D11001223FF021D1822F56222E55BB4C80302FB
:101D21001D254032B4FA03021D2D502BE54C75F0F0
:101D310003246084E5F0B4001DE54C75F060246077
:101D410084E5F0FAC374609A75F00284F5F07405C5
:101D5100A4202402F56222E54C75F003246084E599
:101D6100F0B40018E54C75F060246084E5F075F07E
:101D71000284F5F07405A4202402F56222E55BB427
:101D8100C803021D884019B4FA03021D9050127451
:101D910020C3954D75F008A412236B302402F5621F
:101DA10022E54D75F008A412236B302402F562225E
:101DB100202406E54CFB021DDCE54D75F003A4FB78
:101DC100021DDC20240EE54C75F0038475F002A49D
:101DD100FB021DDCE54D75F002A4FB858232858393
:101DE1003375340075350078328B367537007936A6
:101DF100122288868208868322E572C2E0C2E1C28D
:101E0100E2C2E3C4B40004121E2222B40104121E71
:101E11005A22B40204121E9222B40304121ECA22D0
:101E210022E572C2E4C2E5C2E6C2E7B4000490252D
:101E3100C322B401049025CF22B402049025DB22F1
:101E4100B403049025E722B404049025F322B405D9
:101E5100049025FF2290260B22E572C2E4C2E5C25E
:0E1E6100E6C2E7B4000490261722B4010490F4
:101E6F00262322B4020490262F22B4030490263B8B
:101E7F0022B4040490264722B405049026532290DE
:101E8F00265F22E572C2E4C2E5C2E6C2E7B40004EF
:101E9F0090266B22B4010490267722B40204902678
:101EAF008322B4030490268F22B4040490269B222D
:101EBF00B405049026A7229026B322E572C2E4C28D
:101ECF00E5C2E6C2E7B400049026BF22B401049035
:101EDF0026CB22B402049026D722B403049026E323
:101EEF0022B404049026EF22B405049026FB22901E
:101EFF00270722E572C2E4C2E5C2E6C2E7B40004D6
:101F0F0090000022B4010490000C22B4020490004F
:101F1F001822B4030490002422B404049000302249
:101F2F00B4050490003C2290004822E56D30E40394
:101F3F00C22822D22822E56B30E403C22922D229FB
:101F4F00220570121F5D121F69900030F022900061
:101F5F002FE004B570037570012290002FE0B5706B
:101F6F000122400122F5702220282290002FE0B498
:101F7F000412121FAE121DB1E559F0A3E55AF0A3DA
:101F8F00E55BF022B40203021FC9022017121FAE35
:101F9F00121DB1E0F559A3E0F55AA3E0F55B22E578
:101FAF0070B4010490003722B4020490009A22B456
:101FBF0003049000FD2290016022E570B40123908C
:101FCF000037121DB1E559F0A3E55AF0A3E55BF018
:101FDF009000FD121DB1E559F0A3E55AF0A3E55BA2
:101FEF00F022B4022290009A121DB1E559F0A3E538
:101FFF005AF0A3E55BF0900160121DB1E559F0A313
:10200F00E55AF0A3E55BF022900037121DB1E559B8
:10201F00F0A3E55AF0A3E55BF090009A121DB1E52D
:10202F0059F0A3E55AF0A3E55BF09000FD121DB146
:10203F00E559F0A3E55AF0A3E55BF0900160121D9E
:10204F00B1E559F0A3E55AF0A3E55BF02220291E74
:10205F0090002FE0B4040E122091121DC4E55CF025
:10206F00A3E569F022B402030220AC0220EA122099
:10207F0091121DC4E0F9A3E0900032F0E990003115
:10208F00F022E570B401049001C322B4020490025F
:10209F000522B403049002472290028922E570B40E
:1020AF00011B9001C3121DC4E55CF0A3E569F0901C
:1020BF000247121DC4E55CF0A3E569F022B4021AD1
:1020CF00900205121DC4E55CF0A3E569F09002894A
:1020DF00121DC4E55CF0A3E569F0229001C3121D47
:1020EF00C4E55CF0A3E569F0900205121DC4E55C40
:1020FF00F0A3E569F0900247121DC4E55CF0A3E57B
:10210F0069F0900289121DC4E55CF0A3E569F02225
:10211F00C2AF790C90001605A2121F0205A2122160
:10212F0033D2AF22E0A343D20205A2F0A375D2525D
:10213F0075D2A2E5D220E0FB53D2FD05A2D9E5224C
:10214F00C2AF790C121F0205A290001605A2122130
:10215F0063D2AF2243D202438E20E0A353D2FD536A
:10216F008EDF05A2F0A305A2D9EA22C2AF790C7BBC
:10217F0000121DFA05A290001605A2122190D2AFEF
:10218F0022EB9305A2F0A305A20BD9F522E56BF480
:10219F0030E163E56AF430E45D7405120CE8120275
:1021AF003612023612023612023612023612023678
:1021BF00120236C2AF12220612221812222812223F
:1021CF0038122248122258122268122278D2AF12E5
:0E21DF00023612023612023612023612023692
:1021ED00120236120236120236120236120236125E
:1021FD00023612023612023622790C7B009025B778
:10220D0005A290001605A212219022790C900016BD
:10221D0005A290000005A212213322790C90001620
:10222D0005A290000C05A212213322790C90001604
:10223D0005A290001805A212213322790C900016E8
:10224D0005A290002405A212213322790C900016CC
:10225D0005A290003005A212213322790C900016B0
:10226D0005A290003C05A212213322790C90001694
:10227D0005A290004805A212213322E627F5270872
:10228D0009E637F528782722C3E697F5270809E6EA
:10229D0097F5287827228627872908098628872AEF
:1022AD00122328782C22862C08862D08862E088647
:1022BD002F872909872A1222CB7827792E2275306C
:1022CD000075311012230D1222DE122301D531F4C7
:1022DD0022C3E52E9529E52F952AE530940050016E
:1022ED0022E52E9529F52EE52F952AF52FE530942B
:1022FD0000F53022B3E52733F527E52833F52822FD
:10230D00C3E52C33F52CE52D33F52DE52E33F52EC8
:10231D00E52F33F52FE53033F53022E5278529F00C
:10232D00A4F52C85F02DE528852AF0A4F52E85F051
:10233D002FE5288529F0A4252DF52DE52E35F0F571
:10234D002EE52F3400F52FE527852AF0A4252DF550
:10235D002DE52E35F0F52EE52F3400F52F22B4F0B6
:10236D000122400274F022B47801224002747822D6
:10237D00B43001224002743022900010E004B410F9
:10238D00027400F0900000A98229F582E0229000ED
:10239D0014E0FA900011E004B40F0274FFF09025E0
:1023AD0097932A900014F0900013E004B410027477
:1023BD0000F0F9900014E0FA900000E58229F58212
:1023CD00EAF022900014E0FA900012E004B4110239
:1023DD0074FFF09025A6932A900014F01223B422D6
:1023ED0012238654016008122386541F2460227420
:1023FD007F2212238675F0058412237D243022124C
:10240D0023865401600D12238675F0058412237DF9
:10241D0024302212238675F0058412237D24602238
:10242D00E56C20E210D22430320FC282D287C2B6C0
:10243D00D280C23222C224D232223009120542E5A4
:10244D0042B4FF0B0543E543B4FF04C208C20922A1
:10245D000540E540B4FF190541E541B4FF12754053
:10246D00FF7541FF753CFF753DFF8540488541492E
:10247D0022E56C30E103C20A22200A13D20A300988
:10248D0006C20912257622754200754300D2092233
:10249D00E56C30E003C20B22200B48D20B30240434
:1024AD00C287D282E555240275F00284E5F0B400AE
:1024BD001885404885414975400075410085483C67
:0E24CD0085493D85483E85493F754F00754E57
:1024DB0000054D05551224F1D200D201302406120D
:1024EB001F7702205C22E555B4100E755500754D13
:1024FB0000302405C2A2121F5022E56C30E703C244
:10250B000622200608D206D226D2B6C2A222E56B3C
:10251B0030E703C20722200708D207D226D2B6C261
:10252B00A2222024012220260122754000754100A1
:10253B0085483C85493D85483E85493F7555007525
:10254B004F00754E00754D00757001C22622302468
:10255B00012220260122754200754300854A4485DD
:10256B004B45754C00757001C2262285423285435E
:10257B003375340075350078327536187537007938
:10258B00361222B3864A08E604F54B2203002C0CC4
:10259B0001057E2133E6FF0B4D68146405150D5ABA
:1025AB004B1B26351E1A96114042C8D5000102035B
:1025BB000405060708090A0B008102830405860738
:1025CB0088098A0B008182830485860788898A8B18
:1025DB00008182830485860788098A8B0081828328
:1025EB000485860788898A0B008182830485068788
:1025FB0088898A0B008182838405868788890A8B68
:10260B00008182030485860788090A8B00810203F7
:10261B008405860708898A0B0081020384058607D7
:10262B0008890A8B008182038485860788898A8BB7
:10263B00008182038485860788098A8B0081820347
:10264B008485860788890A8B0081820384850687A7
:10265B0088890A8B008182038405060788890A8B87
:10266B00008102038405860788090A8B0001820317
:10267B008405860708890A8B008102830485060777
:10268B0088098A0B008102038405068708098A0BD7
:10269B00008102830405860788090A8B0081028367
:1026AB000485068708890A8B0081028384058607C7
:1026BB0088890A8B000182830405860708890A8BA7
:1026CB00008102038405060708898A0B0001820337
:1026DB008485860708898A8B000182830405860717
:1026EB0008898A0B008102830405860708890A8BF7
:1026FB00008102030485060708098A0B0001820387
:10270B000485060788090A8B464C414D45205441E8
:10271B004D45204D414348494E45204555524F208C
:10272B005241434B2056455253494F4E202D203298
:10273B003030392D323031322056455253494F4EBD
:10274B0020312E303420286329627920616D706529
:02275B007265A5
:00000001FF
